:10000000C80C0020C5000000C1000000C1000000B5
:1000100000000000000000000000000000000000E0
:10002000000000000000000000000000C10000000F
:100030000000000000000000C1000000C10000003E
:10004000C1000000C1000000C1000000C1000000AC
:10005000C1000000C1000000C1000000C10000009C
:10006000C1000000C1000000C1000000C10000008C
:100070001148000005470000C1000000C100000059
:10008000C1000000C1000000C1000000C10000006C
:10009000C1000000C1000000C1000000C10000005C
:1000A000C1000000C1000000C1000000C10000004C
:1000B000C1000000C1000000C1000000C10000003C
:1000C000FEE7C04610B5154B154A9A420ED2154BA5
:1000D000124A0332D21A92080132920000231048C9
:1000E0001149CC58C45004339342FAD10F4B104AF3
:1000F0009A420ED20F4B0D490331C91A89080131BA
:1001000089000023140000201A19106004338B4268
:10011000FAD104F0BDFC02F065FE10BD0C00002019
:1001200000000020040000203C4F0000C808002010
:100130000C0000201000002070B584B004006A4656
:100140000E4B694661CB61C11B680B600C4B1B6891
:1001500001930C494B699B019B0F9B00985889693F
:100160000905090F013104F0DFFC4000210004F013
:10017000DBFC01304008023804B070BD604E000066
:10018000000000200002005001220A4B1A700022D9
:100190000949180053009B189B00CB189B7ADB077A
:1001A00003D503780133DBB203700132202AF1D189
:1001B0007047C046A4040020A80400200F23034079
:1001C00018003730092B01D8303318007047C0466B
:1001D0000022C30700D55E32830701D5BC235A40F5
:1001E000430701D561235A40030701D5C2235A4072
:1001F000C30601D59D235A40830601D523235A40C7
:10020000430601D546235A4043B2002B01DA8C2322
:100210005A4010007047C04630B5154B1B78002B74
:1002200005D0144B1B780020002B09D119E0124B8C
:100230001B78692B1BD0104B1B78492BF1D116E092
:100240000E4A802109040C4D0A4C93690B42FCD1E3
:100250002B5CDBB213600130C0B22378DBB2834287
:10026000F3D80022034B1A700132054B1A6030BDDF
:1002700076060020B1010020BC01002000000540EE
:100280009442005070B5114B1B78002B1DD1104BC0
:100290001B78002B13D000200E4A802109040E4C3D
:1002A00000260B4D93690B42FCD1235CDBB213603B
:1002B00026540130C0B22B78DBB28342F2D8002240
:1002C000034B1A700132054B1A6070BDF802002012
:1002D000B1010020000005408C0000209442005035
:1002E000184B1B78002B2CD1420883085340434005
:1002F000C208534002095340420953408209534007
:10030000C209534001221340DB011818C0B20E4944
:10031000802212048B691342FCD10B4BDA68102146
:100320008A43DA60D96820220A43DA60D968082251
:100330000A43DA6018601900802252058B69134263
:10034000FCD070479801002000001540F0B55F46D2
:1003500056464D464446F0B491B0444B5D78EDB2FC
:10036000EB1E0020392B79D82C1D002200233F489A
:10037000815C6E46B1540133DBB21A1EA242F7DB38
:10038000AF1C01240020394E335D5840C0B2FFF746
:100390001FFF0134A742F7D12B006B44987003353F
:1003A000012D43DD012300210122314883463148DC
:1003B0008246D946D0465F46D4466846C05CFE2891
:1003C0000FD148460078C0184018FD2446463454E2
:1003D0000131C9B248460078C01840181F3C345457
:1003E00017E0FD280FD122480078C0184018FD24DE
:1003F000204E34540131C9B21D480078C01840184D
:10040000203C345405E05C462478E41864185646D1
:1004100030553878C3185B18053300206446E05423
:100420000132D2B2131EAB42C7DB02E0012300212E
:1004300001220F480478E4B20E4DFE262E550478B2
:10044000E3185B18EE5403780133D2188918C9B247
:1004500001700122084B1A600078C0B211B03CBC98
:1004600090469946A246AB46F0BDC046BC0100206E
:10047000B10100208C00002094420050F0B55F468E
:1004800056464D464446F0B485B0E14B1B78002BF0
:1004900007D0E04B1B68002B03D0FFF7F3FE00F002
:1004A000C0FCDD4B1B78002B00D117E2DB4B1B7827
:1004B000002B00D192E001270024002500230193A6
:1004C000D74B9846D74B9946220000E00F007C1E80
:1004D000E4B26300D449595A4046185A4140404654
:1004E00019521B5A9BB2002B03D1D04B1B78002B07
:1004F0006AD0019B0133DBB20193CD4B1B78002BFB
:1005000048D06E0076197600F31C9A46601C0011E4
:10051000C0B2FFF753FE4B4652469854331D9A46DD
:100520003800FFF74BFE4B46524698546400BE4BD2
:10053000E35A1B0A9A46731D9B4653461809FFF758
:100540003DFE4B465A469854B31D9B465046FFF716
:1005500035FE4B465A469854B34BE45AE4B2F31D69
:100560009A462009FFF72AFE4B4652469854082324
:100570009A46B2442000FFF721FE4B46524698545B
:1005800009360D234A4693556A1C5300D21852006F
:10059000D2B217E06B005B199A1CA2498F54D91C88
:1005A0006400A14AA25A120A9E484254191D9E4A4A
:1005B000A25AD2B2425405330D22C2546A1C5300CF
:1005C000D218D2B20135EDB2944B1B78DBB2791C54
:1005D000C9B2BB4200D979E7140002E0002400232D
:1005E00001938E4B5B78002B00D1A0E0002000230C
:1005F000994600258F4B9A46A0462C006B008E4AE8
:100600009A5A5146595A4A4051465A525B5A9BB2DD
:10061000002B03D1854B1B78002B6DD0019B013340
:10062000DBB201937D4B1E780136AE19F6B2804BDA
:100630001B78002B42D04B465F004F447F00FB1CD1
:1006400043449B463009FFF7B9FD764B5A46985410
:100650003B1D43449B463000FFF7B0FD714B5A46AB
:10066000985463009B46744B5A46D65A360A7C1DF2
:1006700044443009FFF7A2FD6A4B1855BC1D4444A1
:100680003000FFF79BFD674B18556B4B5A46D45A09
:10069000E4B2FE1D46442009FFF790FD614B9855DA
:1006A0003E00083646442000FFF788FD5D4B985514
:1006B000093747440D235B4AD35518E04B465B008E
:1006C0004B449A1C424457498E54DA1C42446400FD
:1006D0005949615A090A534881541A1D42445649DE
:1006E000615AC9B28154053343440D22C2544B466A
:1006F0000133DBB2994601200135EDB2474B5B78FF
:10070000DBB2AB4200D978E7444600280FD0484B13
:100710001B78002B06D04B465B004B445B00E41873
:10072000E4B204E04B465B004B44E418E4B23B4BBC
:100730009B78002B00D1AAE00023994600263F4B6E
:100740009A46A046340073003D4A9A5A5146595A77
:100750004A4051465A525B5A9BB2002B04D1334B4C
:100760001B78002B00D18AE0019B0133DBB201939F
:100770002A4B1B78294A5578ED1801357519EDB2C9
:100780002B4B1B78002B5DD04B465F004F447F0006
:10079000FB1C43449B462809FFF710FD214B5A469A
:1007A00098543B1D43449B462800FFF707FD1D4B13
:1007B0005A46985463009B46214B5A46D55A2D0AF7
:1007C0007C1D44442809FFF7F9FC164B1855BC1D45
:1007D00044442800FFF7F2FC124B1855184B5A46B8
:1007E000D45AE4B2FD1D45442009FFF7E7FC0D4B48
:1007F00058553D00083545442000FFF7DFFC094B04
:100800005855093747440D23064AD35533E0C046AF
:10081000B1010020C0080020F8020020B80100202B
:100820007C060020BC010020540100203F03002072
:10083000CD000020D000002064030020080200202A
:10084000340600204B465B004B449A1C4244D4497A
:100850008D54DA1C42446400D249615A090AD048D6
:1008600081541A1D4244CF49615AC9B2815405339B
:1008700043440D22C2544B460133DBB29946013644
:10088000F6B2C94B9B78DBB2B34200D95AE7C74BEB
:100890001B78002B12D0019D2809FFF78FFCC04C5C
:1008A00060702800FFF78AFCA0706B00AC466344C0
:1008B0005B000433DBB2BE4A137009E0B84B019908
:1008C00059700B0001335A009B18DBB2B84A137001
:1008D000FFF7A2FC0022B74B1A70A2E2B64B1B78BE
:1008E000002B00D19DE2B54B1B78002B00D198E284
:1008F000B34B1B78002B00D193E2B24B1B78002B3B
:1009000000D18BE22027402660250024A64B984684
:10091000AC4B9B4643461B785A461278DBB2934257
:1009200000D9B8E0A1466200A74BD35AA749525A52
:100930005A40102300210120104201D00131C9B2D8
:100940005208013BDBB2002BF6D1A14B1B78002BE8
:1009500006D0A04B1A680123484683401A4201D1B1
:10096000012938D98E4BFE221A70F63A5A709F70C0
:100970000022DA70984A94464946525CD2B29246B6
:10098000511CC9B260464A46815452461A71A2228D
:100990005A7100229A711022DA718C494A4650002D
:1009A000425AD2B21A72425A120A5A72FFF7CEFC57
:1009B0007F4B1870894B1B78002B09D085490A683A
:1009C00001234846834013430B600022844B1A8066
:1009D000FFF758FC5FE04B465B007B4A9A5A7B4925
:1009E000585A504057D08446C30712D401220123DD
:1009F0009A460194010008001041544604420BD16C
:100A00000133DBB20132102BF5D103936046019C18
:100A100005E00023039302E003936046019CFE215E
:100A20005F4B1970F93959709F700021D9706A496C
:100A30008A464B46C95CCBB2019301336A46D372F6
:100A4000D37A9C465346494662465A54544A6B46AA
:100A50001B7913714A005D49525A1040421E904161
:100A6000A122101A4E4A50716B461B7B9371FFF7FF
:100A70006DFC4F4B1870594B1B78002B09D0554912
:100A80000A6801234846834013430B600022544BFD
:100A90001A80FFF7F7FB444B5B784A4A1278DBB2C7
:100AA000934200D9E6E0A14662004E4BD35A4E492C
:100AB000525A5A40102300210120104201D0013126
:100AC000C9B25208013BDBB2002BF6D1404B1B7878
:100AD000002B06D0454B1A680123484683401A4232
:100AE00001D101293AD92E4BFE221A70F63A5A70DA
:100AF0009E7000229446DA7049462031364A92466A
:100B0000525CD2B20192501CC0B2524650546A4656
:100B100012791A71A2225A7162469A711022DA7100
:100B200031494A465000425AD2B21A72425A120A07
:100B30005A72FFF70BFC1E4B1870284B1B78002BCA
:100B400009D02A490A6801234846834013430B60B1
:100B50000022234B1A80FFF795FB8BE04B465B008E
:100B6000204A9A5A20495B5A5A4000D182E0944662
:100B7000D30712D4012101239A46019410000200E8
:100B80000A415446144233D10133DBB20131102BF8
:100B9000F5D103936246019C2DE0002303932AE0E4
:100BA000BC01002034060020B8010020CD00002048
:100BB000B10100203F030020A50400207C0000209C
:100BC000B0010020990100207C0600205401002083
:100BD0003006002004020020940200202B06002092
:100BE00000020020D00000206403002088000020C4
:100BF00003936246019CFE208D4B1870F9385870A3
:100C00009E700020D870484620308A4B9C460300D6
:100C10006146085CC1B2019101316846C172C17A76
:100C20008A4661465046C854814B69460979197114
:100C30004B4659008048095A0A40511E8A41A12159
:100C40008A1A7B494A716B461B7B8B71FFF77EFBCF
:100C50007A4B18707A4B1B78002B09D079490A68B7
:100C600001234846834013430B600022764B1A80D1
:100C7000FFF708FB754B9B78754A1278DBB29342FD
:100C800000D9BDE0A1466200724BD35A7249525A54
:100C90005A40102300210120104201D00131C9B275
:100CA0005208013BDBB2002BF6D16C4B1B78002BBA
:100CB00006D06B4B1A680123484683401A4201D183
:100CC00001293AD95A4BFE221A70F63A5A709D7091
:100CD00000229446DA7049464031564A9246525CA8
:100CE000D2B20192501CC0B2524650546A46127998
:100CF0001A71A2225A7162469A711022DA7156490B
:100D00004A465000425AD2B21A72425A120A5A72D3
:100D1000FFF71CFB494B1870494B1B78002B09D07F
:100D20004F490A6801234846834013430B60002261
:100D3000454B1A80FFF7A6FA62E04B465B00454A36
:100D40009A5A45495B5A5A405AD09446D30712D40E
:100D5000012101239A460194100002000A415446E1
:100D600014420BD10133DBB20131102BF5D10393C7
:100D70006246019C05E00023039302E00393624670
:100D8000019CFE202A4B1870F93858709D70002085
:100D9000D87048464030274B9C4603006146085CAB
:100DA000C1B2019101316846C172C17A8A46614679
:100DB0005046C8541E4B6946097919714B46590073
:100DC0002548095A0A40511E8A41A1218A1A184908
:100DD0004A716B461B7B8B71FFF7B8FA174B187083
:100DE000174B1B78002B09D01D490A680123484680
:100DF000834013430B600022134B1A80FFF742FA23
:100E00000134E4B2124B1B78DBB20135EDB201368E
:100E1000F6B20137FFB2A34200D97BE50022114BA5
:100E20001A7005B03CBC90469946A246AB46F0BD50
:100E3000BC0100209402002064030020B1010020C6
:100E40002B0600208800002000020020B8010020AE
:100E500099010020080200203406002030060020FE
:100E60009C0100201001002070B50400FFF78CF9F0
:100E70002D4A13780133DBB213701378002B03D1A2
:100E800013780133DBB213702849FE230B70F23B59
:100E90004B7000238B7026480378DBB25A1CD2B209
:100EA0000270CB70204B1B78DBB24B71651CEDB22E
:100EB0008D71204B620010198000C05CC87112193E
:100EC00092009B185A780A729A784A721A798A7232
:100ED0005A79CA729A790A73DA794A739B7ADB076C
:100EE00002D58D220A710AE08C22104B1A71630020
:100EF0001B199B000F4AD31800229A725A60630094
:100F00001C19A4000B4B1C19A37A04229343A3724F
:100F1000FFF71CFA084B1870FFF7B4F9074B1D7068
:100F20008022074B1A7070BD2E060020BC010020E5
:100F3000BB010020A8040020B10100202D060020E4
:100F400028060020F8B5FFF71FF9244B1B78DBB209
:100F50000024012B03D800232148002117E0214D54
:100F60002F00012663001B199B00EB189B7ADB07FF
:100F700009D563001B199B00FB189A7AB2439A7239
:100F80002000FFF771FF0134202CEBD1E3E75A007A
:100F900011520133FF2BFAD10023134A1370134A65
:100FA0001370134A1370134A1370134A13801000FE
:100FB0001249134A01240BE093681C4208D093683D
:100FC000234393600C4B1B8801339BB20A4D2B804B
:100FD00003889BB28B42EFD9F8BDC046A404002021
:100FE000BC060020A8040020C408002098010020AE
:100FF000C6080020290600203C0300202F750000B1
:1010000020000140F0B55F4656464D464446F0B4D8
:1010100089B0E04B1B78DBB2DF4AD35CDBB2FE2B3E
:1010200001D001F02FFEDB4ADB4913780133DBB23C
:1010300013701378DBB2CB5CDBB2FE2BF5D001F082
:1010400021FE5A1CD1B22278D318DBB2C25CD2B2D4
:10105000FE2A02D00B1EF4D101E0002906D10023A4
:10106000CC4A1370CD4A137001F0AEFEC94A13701A
:10107000C84A13780133DBB213701378DBB2C64968
:10108000CB5C0233DFB21278D219C44B1E78C44B4A
:101090001B78002B01D00136FF36B046BD4B1B78C4
:1010A000F31A022B00DC81E0BA4B1978C8B21B7826
:1010B000F31A002B01DC01F087FE030000210191EF
:1010C000B54CB44D944632000600E15CC9B2FE292D
:1010D00007D1591EB048415CC9B2FD2901D0012198
:1010E00001910133DBB22978981BC0B2511A8842B2
:1010F000EBDB62464646019B002B01D101F064FE0A
:10110000002354E0B24201D301F05EFEBB420DD297
:10111000FF212278D2180A40825CD2B2FD2A01D186
:101120000137FFB20133DBB29F42F2D84A46127850
:10113000B9B28A46BA18FF25154041464D5D002DCB
:1011400009D1013A92B2FF35154093494D5D002D0A
:1011500001D101F039FEFF252A4001998A5CD2B203
:10116000FE2A33D05A461278013A5244FF210A40EF
:1011700089498A5C0137BF18FFB25A461278D219E2
:1011800096421CD80AE00B78DBB25A1CD2B20A7025
:10119000C35CDBB2FE2B04D101F016FE7D4C2100B6
:1011A0007D4823789E42EED801F00EFE00237A4956
:1011B0008C46784C0800A14680460190A346FF214A
:1011C00011406546695CC9B2FE299BD1714B1B7801
:1011D000013BDBB200227049CA54714B1A70002FD8
:1011E00054D0002301936B4A94468B4660460E0010
:1011F0006C4D6D4A9046A946C24662461278D2B2FC
:1012000059468A5CD2B2FD2A12D1674A1278002A66
:101210000ED10121644A1170013BDBB25D4C227892
:10122000D2B2511CC9B2217000245B498C5428E011
:101230001C000278D2B2B25CD2B2EA540278D2B2C6
:10124000511CC9B201700021B154EA5CD2B2FE2A2D
:1012500006D1019ABA1A013A934201DA01F0B4FDBB
:1012600042461278002A0CD04A46115DF0220A4309
:1012700049460A55002251460A70019A0132D2B2FB
:1012800001920133DBB29F42B7D801E00023019302
:10129000404A137801981B1ADBB213701378DBB243
:1012A000591CC9B2117000213B4AD154831CDBB2D6
:1012B0000693002305933D4B68330793394B5B78C6
:1012C000002B01D000F040FD394BFE221A700022A5
:1012D0009A70344BDB78DBB2312B01D900F013FD6F
:1012E0009B00344AD3589F462E4B9A790023002AFC
:1012F00001D000F025FC00F02EFC2F4900230B70DC
:101300002B4B05225A700A78D2B2501CC0B208701A
:10131000DA7081221A717D325A714F3A9A71FFF751
:1013200015F8264B187000F0EEFC0023244A1370C9
:10133000244A137000F0E7FCFEF726FF22490A78E2
:1013400048788B782149097882189B18CB18DBB232
:10135000164A1370164904224A70174C2278D2B2EA
:10136000501CC0B22070CA7088220A71184A1178C5
:101370000022002900D01A000D4B5A71FEF7E6FF3B
:101380000E4B1870094A002353709370114A137062
:1013900000F0B9FC75060020A403002085000020A1
:1013A00084000020540200202C0600200C000020A5
:1013B000BC010020BC4C0000BB010020B10100209A
:1013C0002D06002028060020B8010020A4040020DB
:1013D000420300204A030020E64B9A781B78934290
:1013E00000D8E4E0E44B1B78002B04D1E2490B78F1
:1013F0000133DBB20B70002A00D1B1E0DD4B5B782A
:101400001F2B29D85A00D2189200DC498A18927AE8
:10141000D20719D501F07EFC581CC0B25900C9187A
:101420008900D64CA4466144897AC9070FD5D149B1
:101430004B705900CA189200A218917A0420814377
:1014400091721F2B5BD907E00133DBB200E0030090
:10145000202BE1D1C74A5370C94B1B78C94A127877
:10146000DBB22020934204D8C54B187840231B1AC6
:10147000D8B2C44B1A78D2B2C1490B784978CB188C
:101480009A4206DBBE4A13785078C01860231B1AB4
:10149000D8B2BD490C234B70BC4C2378DBB25A1C2C
:1014A000D2B22270CB7089230B71B34B1B78DBB2A5
:1014B0004B71B44D2B781B18DBB28B714023CB7171
:1014C00000230B723E334B72B14C23681B0E8B72A0
:1014D0008B7A0133DBB28B7222682B78DBB25E1C15
:1014E000F6B22E70120C9B18C318DBB2CB722368B5
:1014F0001B0ADBB20B732368DBB24B7365E0A249B6
:101500000C234B70A1480378DBB25A1CD2B2027094
:10151000CB7089230B71984B1B78DBB24B71954BC9
:1015200098465B78581CC0B28871944C5E00F218E3
:101530009200125DCA71F2189200A21855780D72CD
:1015400095784D7215798D725579CD7292790A73AD
:10155000F3189B00E318DB794B734346587034E073
:1015600089490C234B7089480378DBB25A1CD2B2EC
:101570000270CB7089230B717F4B1B78DBB24B71F0
:1015800000238B718022CA710B723E334B72804AEA
:1015900013681B0E8B7213681B0CDBB2CB721368C3
:1015A0001B0ADBB20B731368DBB24B730DE0764B97
:1015B00004225A7075480278D2B2511CC9B2017027
:1015C000DA708B221A7174325A71FEF7BFFE714BBA
:1015D0001870684A93780133937094E36A4B05223C
:1015E0005A706A480278D2B2511CC9B20170DA70DE
:1015F00083221A717C3A5A7100229A71FEF7A6FE74
:10160000644B18707FE360490A234B705F4803788E
:10161000DBB25A1CD2B20270CB7084230B71043B34
:101620004B7100238B713E33CB71594A13681B0EEB
:101630000B7213681B0CDBB24B7213681B0ADBB214
:101640008B721368DBB2CB72FEF780FE514B1870C1
:1016500059E34D4B062058704C4C2278D2B2511CA5
:10166000C9B22170DA7085221A71843ADA719871E0
:1016700000225A71FEF76AFE464B187043E3424B54
:1016800004225A7041480278D2B2511CC9B201708A
:10169000DA7082221A71404A1279D2B25A71FEF778
:1016A00055FE3C4B18702EE300233C4A13703C4A15
:1016B0001360EEE201233B4A1370384A1370384A34
:1016C0001360394A1370E4E22F4B04225A702F48FA
:1016D0000278D2B2511CC9B20170DA7092221A712A
:1016E000903A5A710022234BDA70FEF72FFE294BF5
:1016F000187008E3284B1B79DBB2FC2B05D0FD2BBF
:1017000007D100221B4BDA700AE00122194BDA7074
:101710001BE0184BDB78002B02D0012B46D114E0E4
:10172000194B05225A7019480278D2B2511CC9B21D
:101730000170DA7090221A716D325A71F53A9A710D
:10174000FEF704FE134B187044E00F4B05225A704D
:101750000E480278D2B2511CC9B20170DA709022E0
:101760001A716C325A71E43A9A71FEF7EFFD094B27
:1017700018702FE00C0000202E060020A804002086
:10178000B80100204A030020BC010020BB0100205A
:1017900078000020B101002054020020A5040020A0
:1017A000C0080020B001002010010020D94B042205
:1017B0005A70D9480278D2B2511CC9B20170DA709D
:1017C00091221A71D54A1279D2B25A71FEF7BEFD32
:1017D000D34B1870D34AD3780133D37093E2D24BF2
:1017E0001B78002B05D00023CF4A1370CF4A13601B
:1017F00002E00122CC4B1A70C64A04235370C6483B
:101800000378DBB2591CC9B20170D37087231371FE
:10181000C54B1B78591E8B41DBB25371FEF796FD09
:10182000BF4B18706FE2BB4B04225A70BA48027863
:10183000D2B2511CC9B20170DA708A221A710A3A06
:101840005A71FEF783FDB64B18705CE2B84B1B78FB
:10185000002B00D157E2B14B1C79E4B2092C04D91A
:101860000022B34B1A7001F0AFFA611DAB4B5D5C07
:10187000EDB2092D04D90022AD4B1A7001F0A4FA83
:10188000631DEB18DBB2A34A5370A34E3378DBB26F
:10189000581CC0B23070D370932313719F4B1B79C7
:1018A000DBB25371002C12D0621ED2B20632052375
:1018B0009A488446974E8846581C6146CB5CDBB2FA
:1018C000335403008242F7D14146230000E0230055
:1018D0000633924A525CD2B28E49CA54002D01D1CD
:1018E00001F0E5F9A31D691EC9B2E21D89188B4EEE
:1018F00088485A1CF35CDBB28354131E8B42F8D128
:10190000FEF724FD864B1870844B5A79303AD2B2D8
:10191000012C0ED906200121804E9300D2185200CE
:10192000335C303BD218D2B20131C9B201308C42A3
:10193000F3D8A31D7949CB5C303BDBB2012D0FD925
:10194000E01D023DEDB208342C190D0099005B1822
:101950005B00295C30395B18DBB201308442F5D181
:10196000032A00D9CFE1191C322B00D93221013AC8
:10197000704B99540122704B1A70C4E16C4B1B7868
:10198000002B00D1BFE1654B1C79E4B2092C04D9CE
:101990000022674B1A7001F017FA604B5B79303BFD
:1019A000DBB2012C0ED9A01EC0B2073006215B4D60
:1019B0009A009B185B006A5C303A9B18DBB20131DD
:1019C0008842F5D122000832D2B252484270524DBC
:1019D0002A78D2B2511CC9B22970C2709322027106
:1019E0004E4A1279D2B24271002C0CD0611EC9B29B
:1019F00006310522494E0500501CB25CD2B22A5471
:101A000002008142F8D1A21D032042498854032BD1
:101A100021D8E21D0E003021B154013B454AD05C73
:101A2000C0B2343103F006F9CDB208239846A04481
:101A30000A21280003F078F803003033DBB2424675
:101A4000B35409340A21280003F0F4F80B003033B2
:101A5000DBB2335509E0E21D2E4B322199542100AF
:101A6000083135225A5409341A55FEF76FFC2C4BB5
:101A7000187048E100202E4B1870264B04225A7033
:101A8000254C2278D2B2511CC9B22170DA7094224E
:101A90001A715871FEF75AFC214B187033E11F4B35
:101AA000DA79D2B2254B1B681B0E9A4200D02AE18C
:101AB0001A4B1A7AD2B2214B1B681B021B0E9A4298
:101AC00000D020E1154B5A7AD2B21C4B1B681B0484
:101AD0001B0E9A4200D016E1104B9B7ADBB2174ADC
:101AE0001268D2B29A4200D00DE10120104B18705A
:101AF000084B04225A70084C2278D2B2511CC9B249
:101B00002170DA7094221A715871FEF71FFC044B91
:101B10001870F8E0BC010020BB0100205402002036
:101B2000B10100200C0000204B0300209442005023
:101B30002A060020B8010020A6040020780000201A
:101B4000E149E248DA1D8A5CC2540133DBB28A798A
:101B5000D2B29A42F6D80021DC4AD154DA4B0122A3
:101B60005A71DB490A705B79002B04D137E0D64B00
:101B70005B79002B33D0D54B1B78002B01D101F0C2
:101B8000A3F8D44A01231178002906D00133DBB22F
:101B90000132182BF7D101F0EFF8991DC9B2CE4AE6
:101BA0005170CE4C2178C9B2481CC0B22070D1709F
:101BB000952111710021517101319171D371002B67
:101BC00029D0591EC9B209310823C04CC2481A0095
:101BD000083AA25CC25401339942F8D11BE0BE49D5
:101BE0000C234B70BD480378DBB25A1CD2B2027092
:101BF000CB7095230B7100234B718B710633CB7126
:101C000054330B720B334B7210338B72023BCB721B
:101C1000533B0B734B73FEF799FBB14B187072E09B
:101C2000AD4905234B70AD480378DBB25A1CD2B2E4
:101C30000270CB7086230B71AA4B1B78DBB24B7101
:101C400000238B71FEF782FBA54B18705BE000232D
:101C5000A24A1370A44A1370A44A1370A44A1360D2
:101C6000A44A13700121A44A1170A44A13700022DF
:101C7000A34C012053009B189B00E318997A8143E1
:101C800099720132202AF5D103E08F4B1B79002B8A
:101C900039D19C4B00221A70781EC2B25A708A4900
:101CA0000A78D2B29A704A78D2B2DA7002280CDD81
:101CB000022202230D00934C911CAA5CD2B2625402
:101CC0000133DBB21A1E8242F6DB00228E4B1A7001
:101CD0008E488F4A01211D001C000FE093681942B5
:101CE00006D093680B4393602B780133DBB22B70E3
:101CF0002378DBB2142B01D900F053FF0378002BBB
:101D0000ECD100F04EFF704B1B78069A944663446A
:101D10009F4201DC00F092FF6B4B18780130C0B29B
:101D20003F1AFFB2002F01D1FFF7C8FA7C1EE4B2C0
:101D3000013400236449C2188A5CD2B2CA54013308
:101D4000A342F8D1FFF7BAFA5F4B5B78DBB21F2BE7
:101D500001D800F0B7FE5C4B9B78002B01D000F05F
:101D6000B1FE594B5B78DBB25F2B05D9564B5B78E4
:101D7000203BDBB298460FE0534B5B78DBB23F2B46
:101D800005D9514B5B78203BDBB2984604E04E4BC3
:101D90005B78203BDBB298464F4BFE221A704A49D3
:101DA0004A78D2B29A700022DA700B79DBB2252B16
:101DB00001D900F067FE9B00564AD3589F4656490A
:101DC000002342468B54444B06225A7042468A5C9A
:101DD000D2B2501CC0B2444608551A7181225A71C1
:101DE0007D329A714F3ADA71FEF7B0FA3C4B1870B7
:101DF00000F048FE384B06225A7047484246825C43
:101E0000D2B2511CC9B2444601551A7183225A718B
:101E10007C3A9A710022DA71FEF798FA304B18700A
:101E200000F030FE00223D4B1A7000F02BFE012224
:101E30003A4B1A7000F026FE274A0B23537036489F
:101E40004346C35CDBB2591CC9B244460155137109
:101E500084235371443B93710023D3713E33137237
:101E60002F490B681B0E53720B68174840781B0CE8
:101E70001B1A4433DBB293720B681B0ADBB2D372BA
:101E80000B68DBB21373FEF761FA154B187000F0A4
:101E9000F9FD114907234B701F484346C35CDBB271
:101EA0005A1CD2B2444602550B7185234B71002354
:101EB0008B710633CB71053B0B72FEF747FA084B6B
:101EC000187000F0DFFDC046540200204C030020D3
:101ED000780600204D030020BC010020BB0100203B
:101EE000B1010020CC0000207506002085000020F4
:101EF00094010020480300207E00002042030020BF
:101F0000A8040020FC020020740600209801002094
:101F100020000140844D000094020020B001002008
:101F200078000020B34905234B70B3484346C35C97
:101F3000DBB25A1CD2B2444602550B7182234B715C
:101F4000AE4B5B79DBB28B71FEF700FAAC4B1870CD
:101F500000F098FDAB4B1B78002B05D00023A94A5D
:101F60001370A94A136002E00122A64B1A70A1491E
:101F700005234B70A0484346C35CDBB25A1CD2B267
:101F8000444602550B7187234B719E4B1B785A1E9A
:101F90009341DBB28B71FEF7D9F9994B187000F0C1
:101FA00071FD944B05225A7093484246825CD2B22E
:101FB000511CC9B2444601551A718A225A714A3AD3
:101FC0009A71FEF7C3F98E4B187000F05BFD8B4BD6
:101FD000DB79DBB2102B02D91022884BDA71874BE8
:101FE000DB79002B0DD00023844988481A00083281
:101FF0008A5CC2540133DBB2CA79D2B29A42F5D8B4
:1020000000E000230021814AD15401227B4B9A71C8
:102010001F254545AD416D426B02029343463F2B60
:1020200002D98023DB000293A022D20580235B002B
:10203000592616248820D650D450D050D158002983
:10204000F9D0734B1A6801210A431A602222DA6020
:10205000FD2252025A601961BFF36F8F1A00136993
:10206000002BFCD1FD22520202990B00FA20400203
:102070008446634404930B0066498C4663449B4644
:10208000634B0024012021218A46FE2149028C460F
:10209000B9465E4604990391029FB118DC6059600D
:1020A0009C601861BFF36F8F19690029FCD1996892
:1020B0005546DD605A6099601861BFF36F8F1969EA
:1020C0000029FCD104326245E4D13E004F46504B1A
:1020D0002222DA60039A5A6001221A61BFF36F8FDD
:1020E0001A69002AFCD149480178090643781B0483
:1020F000C91883781B02CB18C1785B1802931F257F
:1021000043461D40424B0121FA2040028146B14422
:102110003E4884464846B946070094B22409A54281
:1021200000D07FE0BC182120D8605C6002989860E5
:102130001961BFF36F8F1C69002CFCD133480479FF
:10214000200683463148447924045C44A2468479BD
:1021500024025444C079824654442F488246B244F3
:1021600092442120D860504658609C601961BFF3AA
:102170006F8F1C69002CFCD12448047A200683460A
:102180002248447A24045C44A246847A24025444BB
:10219000C07A8246544421488246B2449244212067
:1021A000D860504658609C601961BFF36F8F1C69FE
:1021B000002CFCD16046047B200683466046447BAD
:1021C00024045C44A246847B24025444C07B82469F
:1021D000544413488246B24492442120D860504669
:1021E00058609C601961BFF36F8F1C69002CFCD193
:1021F0008AE0C046BC010020940200205402002066
:10220000B10100204B03002094420050A0010020A7
:1022100000C0005000FAFFFF04F4010008F40100C0
:102220000CF401000020D860FD24640214195C60E5
:1022300098601961BFF36F8F1C69002CFCD19C68FA
:10224000A246BC182120D8605C6050469860196195
:10225000BFF36F8F1C69002CFCD10020D860D748D9
:1022600014185C60002098601961BFF36F8F1C69BF
:10227000002CFCD198688246D1483418A41821203B
:10228000D8605C60504698601961BFF36F8F1C691D
:10229000002CFCD10020D860CA4814185C600020D3
:1022A00098601961BFF36F8F1C69002CFCD198688E
:1022B0008246C5483418A4182120D8605C60504676
:1022C00098601961BFF36F8F1C69002CFCD100204E
:1022D000D860BE4814185C60002098601961BFF394
:1022E0006F8F1C69002CFCD198688246B84834185E
:1022F000A4182120D8605C60504698601961BFF333
:102300006F8F1C69002CFCD110328024A400A242E3
:1023100000D002E74F46AF4A136801218B43136098
:10232000002180235B00A022D205D150AA4B9B79CB
:10233000002B7ED0A022D20580235B0059251624D5
:102340008820D550D450D050D1580029F9D0A14A76
:10235000116801230B4313604046FA256D01454483
:102360002D019E4C10239946A944210000260F3BC5
:1023700098468446D6605560966043461361BFF325
:102380006F8F1369002BFCD19368180E0870180C1E
:102390004870180A8870CB7004350431A945E9D11A
:1023A00060468C4A136801218B431360002180230F
:1023B0005B00A022D205D150884B1B78FF2B05D1A2
:1023C000864B20221A7000225A7007E0002B05D19C
:1023D00000F08DFC6378002B02D108E00121F9E7C1
:1023E0000131C9B201341029F4D100F0D9FCCB1D60
:1023F000DBB27B4C63707B4D2B5CDBB25A1CD2B2E0
:102400002A542371952363710023A3710133E3716F
:10241000217200294AD00139C9B20A3109236F4C0F
:102420006F481A00093AA25CC25401338B42F8D1BA
:102430003CE06B4C152363706A494346CB5CDBB2CE
:102440005A1CD2B240460A5423719523637100236B
:10245000A371E3710E332372653363723B3BA37246
:10246000E3720B3B2373203363732233A3730B3B61
:10247000E37311332374093B63744C3BA374430926
:102480003133E3742E2323751F2505400A212800CC
:1024900002F04AFB03003033DBB263750A212800E7
:1024A00002F0C8FB0B003133DBB2A375FDF74EFF22
:1024B0004D4B1870E6E24A4B05225A704948424695
:1024C000825CD2B2511CC9B2444601551A719222A3
:1024D0005A718C3A9A71454B0433002207991A704D
:1024E00001339942FBD1FDF731FF3F4B1870C9E230
:1024F000394B5B78DBB23F2B04D8374B5B78203B02
:10250000DBB215E0344B5B78DBB25F2B07D8324B84
:102510005B78374A1278D318403BDBB208E02E4B89
:102520005A7833490B7849789B18603BCB18DBB25B
:10253000294A5279D2B2022A16D004D8002A09D0E8
:10254000012A0CD023E0FC2A1DD0FD2A16D0032A34
:102550001DD10EE0254AD31800221A7117E0234A34
:10256000D31801221A7112E0204AD31802221A71DC
:102570000DE01E4AD31803221A7108E01B4AD31833
:1025800004221A7103E0194AD31805221A71124B5A
:102590005B78DBB23F2B04D80F4B5B78203BDBB280
:1025A00031E00D4B5B78DBB25F2B23D80A4B5B78B5
:1025B0000F4A1278D318403BDBB224E004FA010042
:1025C00004F4010008FA010008F401000CFA01000B
:1025D0000CF4010000C0005054020020A0010020B3
:1025E000BC01002094020020B10100200C0000205A
:1025F000B8010020E44B5A78E4490B7849789B18DD
:10260000603BCB18DBB21900E14AD2181279052AD7
:1026100000D9ACE09200DF4B9B589F46DE48062372
:102620004370DE4C4346E35CDBB25A1CD2B24546F3
:102630006255037190234371002383711033C3717A
:10264000D34B5B1801221A71FDF780FED44B187032
:1026500018E2D14806234370D04C4346E35CDBB21A
:102660005A1CD2B2454662550371902343718F3B89
:102670008371CC4B1A78531E9A41D2B2C271C44BAB
:102680005B1802221A71FDF761FEC54B1870F9E163
:10269000C14806234370C14C4346E35CDBB25A1C7D
:1026A000D2B2454662550371902343718E3B8371CC
:1026B000013BC371B64B5B1803221A71FDF746FE4E
:1026C000B74B1870DEE1B44806234370B34C434661
:1026D000E35CDBB25A1CD2B24546625503719023CB
:1026E00043718D3B8371B04B1A78531E9A41D2B21D
:1026F000C271A74B5B1804221A71FDF727FEA84B85
:102700001870BFE1A44806234370A44C4346E35C21
:10271000DBB25A1CD2B24546625503719023437115
:102720006D338371F53BC371994B5B1805221A71A8
:10273000FDF70CFE9A4B1870A4E1974806244470EC
:10274000964D4346EB5CDBB25A1CD2B24646AA55C4
:102750000371902343716C338371EC3BC3718C4BD9
:102760005B181C71FDF7F2FD8D4B18708AE18A4CE5
:1027700005216170894D4146695CC9B2481CC0B2EF
:102780004646A8552171912161717F494979C9B2A5
:10279000A1717F49CB1801321A71FDF7D7FD804B2B
:1027A00018706FE1784B5B79DBB2012B1BD0002BEB
:1027B00002D0032B3FD067E0774B05225A70774851
:1027C0004246825CD2B2511CC9B2444601551A71CC
:1027D00090225A7100229A711032DA71FDF7B6FD1B
:1027E0006F4B18704EE1684B9B79002B03D0012290
:1027F0006C4B1A7002E000226A4B1A70664906237D
:102800004B7066484346C35CDBB25A1CD2B24446A6
:1028100002550B7190234B7101248C71614B1B7815
:102820005A1E9341DBB2CB71FDF790FD5C4B1870E3
:102830005E4B1C7026E1544B9B79002B03D0012288
:10284000594B1A7002E00022574B1A705249062366
:102850004B7052484346C35CDBB25A1CD2B244466A
:1028600002550B7190234B718D3B8B714E4B1B7836
:102870005A1E9341DBB2CB71FDF768FD484B1870CF
:1028800001224A4B1A70FDE0434905234B7043482F
:102890004346C35CDBB25A1CD2B2444602550B71AC
:1028A00091234B71384B5B79DBB28B71FDF74EFD99
:1028B0003B4B1870E6E0344948798B79DB08C00857
:1028C000181AC0B2831DDBB2334A5370334D4346EE
:1028D000EB5CDBB25C1CE4B24646AC551371A22340
:1028E00053714B79DBB29371C300DBB2D371002813
:1028F00075D004000934E4B209260D003300093B09
:10290000D9B2731EDBB26A78D2B25F2A15D9CA0770
:1029100009D51D4A5278603A52002549525A120A86
:102920001D49CA5453E0184A5278603A520020496F
:10293000525AD2B21849CA5449E0134A5278D2B214
:102940003F2A15D9CA0709D50F4A5278403A520092
:102950001849525A120A1049CA5438E00A4A5278A1
:10296000403A52001349525AD2B20B49CA542EE08F
:10297000CA0723D5044A5278203A52000E49525AC7
:10298000120A0549CA5422E054020020B80100206E
:102990000C0000201C4E0000BC010020940200200E
:1029A000B10100207C0000202B060020A60400209E
:1029B00008020020D00000207C060020DB4A52786C
:1029C000203A5200DA49525AD2B2DA49CA54013690
:1029D000F6B2B44292D10830C3B2059301E00823A5
:1029E00005930023D44A1360D44A1360D44A136079
:1029F000FDF7ACFCD34B187044E0CE4B07225A7065
:102A0000D1484246825CD2B2511CC9B244460155FB
:102A10001A71A9225A7100229A71DA711A72FDF79D
:102A200095FCC84B18702DE0C04B5B78DBB21A00E8
:102A3000203AD2B21F2A09D8BF4803680121914029
:102A40008B4303600022C14B1A7018E03F2A0BD859
:102A5000BA480268403BDBB2012199408A430260D8
:102A60000022BA4B1A700AE0B5480268603BDBB23C
:102A7000012199408A4302600022B44B1A7000225F
:102A8000B04B1A70A94B1B78069A944663449F4238
:102A900000DCD3E0A54B18780130C0B23F1AFFB27A
:102AA000002F01D1FEF70AFC7C1EE4B201340023A2
:102AB0009E49C2188A5CD2B2CA540133A342F8D1EB
:102AC000FEF7FCFBA24A00231370019BFB1ADBB24A
:102AD000537096490B78DBB293704B78DBB2D370AE
:102AE000022F0FD9FC1EE4B2033402230E001100A2
:102AF0000025981CF25CD2B20A545A1D8D54013341
:102B00009C42F6D1924B9B780222069BFB1A90487E
:102B10000EE0815C01315218D2B2111F7C2907D915
:102B200001238B490022CA5401333C2BFBD14BE1DA
:102B30009A42EEDB023AD2B2854B5A700022854BA4
:102B40001A70854D8548012419001A000DE083682C
:102B50001C4206D08368234383600B780133DBB2C9
:102B60000B701378DBB2142B02D82B78002BEED12C
:102B70000022784B1A701800784A01211C0009E0E5
:102B80009368194206D093680B439360237801330E
:102B9000DBB223700378DBB2012BF1D900226D4B3D
:102BA0001A706B4B5C78E4B23F2C47D86C4980229A
:102BB00012048B691342FCD10020FDF791FB684B96
:102BC000D96810220A43DA60D96820220A43DA6001
:102BD000D96808220A43DA60631C99460127012656
:102BE0005F4C80252D045A4B984600239A46A369D2
:102BF0002B42FCD14346DB5DDBB223604346D85D0C
:102C0000059B5840C0B2FDF7E3FA05904346524693
:102C1000DA550136F6B2371E4F45E8DD50498022BD
:102C200012048B691342FCD14D4B059A1A600123A3
:102C300047490022CA5401333C2BFBD1494B1B7836
:102C4000494A1278DBB2934204D10023454A1370FB
:102C5000454A13703B4B1B78002B00D1B4E0FDF7C5
:102C600011FBB1E0404B1B780133DBB23F4AD25C31
:102C7000D2B2FE2A01D1FEF7F9F902233A4C3B48C1
:102C8000FEF7DFF9384A1378013BDBB21370137893
:102C9000DBB2364AD35CDBB2FE2BE3D1FEF7E8F9B8
:102CA0000634224B1B5D303BDBB2FEF759FEFDF7CD
:102CB0004DFB244B18701D4B5A79303AD2B2012C7F
:102CC00001D9FEF727FEEBE71A4B06225A70284877
:102CD0000278D2B2511CC9B20170DA7095221A7111
:102CE00000225A7101219971DA71FEF794FF114B9C
:102CF00007225A70144C225CD2B2511CC9B2215422
:102D00001A7195225A7100229A710121D9711A7291
:102D1000FFF7CCFB5A00D3189B00164AD3189A7AB7
:102D200004218A439A72FEF7EAFBC046540200204F
:102D30007C060020BC010020040200208800002046
:102D40009C010020B10100209402002077060020A1
:102D5000FC020020740600209801002020000140A1
:102D6000000015408500002075060020A403002007
:102D7000BB010020A804002017481E224270174CF7
:102D80002278D2B2511CC9B22170C2709522027150
:102D900000224271013282711732C271FEF711FFB7
:102DA0000D4C172363700E4D2B5CDBB25A1CD2B254
:102DB0002A542371952363710023A3710133E371B6
:102DC0000F332372FFF727FB09B03CBC90469946AE
:102DD000A246AB46F0BDC046BC010020BB010020AE
:102DE00094020020F0B55F4656464D464446F0B486
:102DF00085B0904D904B2B60904C914B2360914847
:102E0000914A026091490B60914A924B13600023F2
:102E1000AB60A360836080338B60703B9360A022C3
:102E2000D205F033592416208821D450D050D150E7
:102E3000D558002DF9D0884A116801230B4313603F
:102E4000864B1100012202E0013B002B02D0C86832
:102E50000242F9D0804B00221A611A6A802149028D
:102E60000A431A627E4A1A627C4B7B49042202E0C2
:102E7000013B002B02D0C8680242F9D0764B0222F7
:102E80001A61784A9A60802252045A6101F0AEFDBC
:102E90000123754A1360754A11680B431360744A25
:102EA000F9214902714B00240126724DDC60596002
:102EB0009C601E61BFF36F8F18690028FCD1986871
:102EC000070E1770070C5770070A9770D0700431FF
:102ED0000432A942EAD1664B1B78FF2B04D1644B24
:102EE00020221A7000225A70604B0022DA60624978
:102EF00059609A6001321A61BFF36F8F1A69002A14
:102F0000FCD15A4B9A685D490A600A681204120C97
:102F10000A600022DA60F821490259609A600132A1
:102F20001A61BFF36F8F1A69002AFCD14F4B9B685F
:102F3000D9B2534A1170DA0503D50121514A1170F3
:102F400002E000214F4A11709B0503D501224E4B30
:102F50001A7002E000224C4B1A70444B0022DA60D7
:102F60004A4959609A6001321A61BFF36F8F1A693A
:102F7000002AFCD13D4A9368116801208143116009
:102F80003E490A6890200006844662440A60D9B22D
:102F90003F4A1170190AC9B251701B0CDBB2937011
:102FA0001378DBB2202B02D90122394B1A70384B2F
:102FB0005B78DBB2202B02D90122354B5A70344B9F
:102FC0009B78DBB2202B02D90122314B9A70304A18
:102FD00013785278DBB2934205D92D4B1B78DBB2C4
:102FE000274A137004E02A4B5B78DBB2244A137043
:102FF000274B9B78224A1278DBB2934204D9244BA8
:103000009B78DBB21E4A13700322A023DB05DA6330
:10301000204B1B68002B43D1023A1F4B1A7096209D
:103020008001FDF789F8C0239B0518431B4B5862AC
:103030003FE0C04600400050F7FF00004040005015
:10304000FFFF00008040005015150000C0400050F8
:103050000041005015FF00000002005091D0030015
:1030600017420000080003009442005000C00050C6
:103070004C03002018F20100FC0F10007800002023
:10308000990100207C0000202B06002004F00100A4
:10309000B80100207C420050F802002000000540EA
:1030A000E1204002FDF748F8C0239B051843DA4BA6
:1030B0005862D94B03229046DA605A6801273A4396
:1030C0005A60D64CC326B600A359FF2293431A0078
:1030D00040231343A35180235B012360A025ED050A
:1030E000C0231B016B63C0239B002B63CC48FDF7FF
:1030F00023F8C0239B051843CA4B58620B22DA60A1
:1031000042461A638022D200DA629A68F0218A432A
:103110009A60002119615A6817435F6080239B0100
:103120002360A259C04B1A40A251C04A11608020AE
:10313000C0041060BE481060BE485060C2229200B9
:10314000A0580340C02000020343A35080235B002B
:10315000E950A73B9B46B84B1B78002B5FD0A022C1
:10316000D20580235B00162088215C46D450D050C5
:10317000D150D458002CF8D0B04B1A6801210A4322
:103180001A602222DA60F82252025A601961BFF3F3
:103190006F8F1A69002AFCD1A94B1B78DBB2A94AB0
:1031A0001278002A02D0802252001343A64A1278D5
:1031B000002A02D0802292001343A04A2121D1602C
:1031C000F82149025160936001231361BFF36F8FAF
:1031D00013001A69002AFCD19C4908784A788B7838
:1031E000120282181B04D318944A2121D1609849F5
:1031F0005160936001231361BFF36F8F13001A694D
:10320000002AFCD18D4A136801218B4313600023EF
:1032100080225200A021C9058B50874A13708D4B24
:103220001B78002B56D0A022D20580235B001620ED
:1032300088215C46D450D050D150D458002CF8D0BE
:103240007E4B1A6801210A431A602222DA60F822B2
:1032500052025A601961BFF36F8F1A69002AFCD1BC
:10326000764B2232DA60F92252025A6001221A6148
:10327000BFF36F8F1A69002AFCD17748F9256D02D8
:103280006E4C21239C460127744E02781206437827
:103290001B04D21883781B02D318C2789B1862468D
:1032A000E2606560A3602761BFF36F8F2369002B25
:1032B000FCD104300435B542E7D1604A13680121DE
:1032C0008B431360002380225200A021C9058B503C
:1032D000604A1370624B1B78624A1278DBB29342E9
:1032E00001D0FDF78FFE604B1B78604A1278DBB28D
:1032F000934200D12CE35C4B1B78002B36D1FF337B
:10330000FF335B4AD35A9BB280225200934222D0B1
:1033100055490B78DBB25A1CD2B20A705B00544A92
:103320009B5A9BB280225200934214D0023A08006A
:103330004F4D802464000378DBB2591CC9B2017080
:103340005B005B5B9BB2A34205D0013AD2B2002A7C
:10335000F1D101F041F9444B1B785B00444A9B5A80
:103360009BB28022520093422ED03BE03E4B1B7812
:10337000013B5B003E4A9B5A9BB280225200934223
:10338000E9D039490B78DBB25A1CD2B20A705B0023
:10339000374A9B5A9BB2802252009342DBD0023ABA
:1033A0000800334D802464000378DBB2591CC9B295
:1033B00001705B005B5B9BB2A342CCD0013AD2B2FE
:1033C000002AF1D101F00CF9274A2948802149004F
:1033D00013780133DBB2137013785B001B5A9BB276
:1033E0008B42F5D0204B1B785B00214A9B5A9BB245
:1033F000002B00D1ACE21C4B1B785B009B5ADBB26C
:103400009A1CD2B2402A02D9FDF79CFDA0E2032A01
:1034100030D8FDF797FD9BE20000054000E100E099
:1034200020A1070000001540FF00FFFF2000014021
:10343000000001685D020000A604002000C00050EA
:10344000990100207C0000202B060020B8010020FC
:1034500004F00100780600204C03002018F201005F
:103460008500002075060020C6080020C408002042
:10347000BC060020DE490978C9B2142908D9DD4903
:1034800009788918C9B249008024A400DA480C528E
:10349000D84909788918C9B24900D748095A89B268
:1034A00080208000814200D052E2D24D297801393B
:1034B000C9B2D148490000240C5229788918C9B2F0
:1034C00049000C52002A01D101F0B2F85C1CE4B2B0
:1034D000013400250020C74FC74B9846C74E3B78A4
:1034E000DBB25A1CD2B23A705B0042469B5ADBB246
:1034F0007355735D5840C0B2FCF76AFE0135AC42AB
:10350000EDD1BC4A13780133DBB21370BB4B1B798E
:10351000DBB2F02B00D08FE1B84B9B78002B00D0B2
:103520008AE1002800D013E2B448047A417A827A12
:10353000C37A0902611812048A181B06D318B04A0C
:103540001360B04C00210022AF4DAD484B005B181A
:103550009B00EB189B7ADB0734D5036826689E42F4
:1035600030D1AA4BFE221A70F33A5A7000229A7098
:10357000A7480278D2B2511CC9B20170DA70862213
:103580001A71743A5A719D4A5179C9B299719179F7
:10359000C9B2D971D179C9B21972117AC9B2597245
:1035A000517AC9B29972917AC9B2D972D27AD2B229
:1035B0001A73FCF7CBFE974B1870FCF763FEFDF710
:1035C000C1FC8BE00132D2B201310C34202ABDD1D2
:1035D0008D4B9B7ADB0701D401F037F801218A4833
:1035E000CAB24B005B189B00C3189B7ADB0701D45F
:1035F00001F02CF801312029F2D16FE053009B1823
:103600009B0081498C4663449B7ADB0703D50132DA
:10361000D2B21F2AF2D9202A07D11F3A7E4B1A7044
:103620007E4C7F4A012021000DE000227A4B1A7067
:10363000F6E79368184206D09368034393600B78CB
:103640000133DBB20B702378DBB2042BF1D90022FB
:10365000724B1A70734B5C78E4B2734A80231B047C
:1036600091691942FCD10020FCF73AFE6E4BD968F3
:1036700010220A43DA60D96820220A43DA60D96846
:1036800008220A43DA601C602000FCF7A1FD013427
:10369000012C17DD02250223634F8022120490467D
:1036A000604EBA6941460A42FBD1F25CD2B23A603E
:1036B000F35C5840C0B2FCF78BFD0135EDB22B1E18
:1036C000A342EEDD584A80231B0491691942FCD1C4
:1036D000554B18600022554B1A6039E1514B0022BE
:1036E0001A700B21597001399970DA701A7172329F
:1036F0005A71424A5179C9B299719179C9B2D97155
:10370000D179C9B21972117AC9B25972517AC9B252
:103710009972917AC9B2D972D27AD2B21A733F4CE5
:103720003F4A0120210009E09368184206D09368BF
:10373000034393600B780133DBB20B702378DBB269
:10374000132BF1D90022354B1A70364B5C78E4B25A
:10375000354A80231B0491691942FCD10020FCF7F3
:10376000BFFD314BD96810220A43DA60D9682022A4
:103770000A43DA60D96808220A43DA601C60200034
:10378000FCF726FD0134012C17DD02250223264F0C
:10379000802212049046234EBA6941460A42FBD168
:1037A000F25CD2B23A60F35C5840C0B2FCF710FD54
:1037B0000135EDB22B1EA342EEDD1B4A80231B0414
:1037C00091691942FCD1184B18600022174B1A60FE
:1037D00000230949580042520133402BFAD10023FB
:1037E000134A1370134A1370024A1370B0E0C046B4
:1037F00029060020C6080020BC0600201401002075
:1038000044030020AC040020A8040020BC010020D8
:10381000BB010020B1010020B2010020740600208D
:1038200020000140FC02002000001540944200509E
:10383000C40800209801002000286BD1BF4B1E78DF
:103840000136F6B201230025FE226946CA73761BB3
:10385000F6B2BB4A6946C97B11705C1CE4B2B74A38
:10386000D55C0135EDB2402D72D8B54A5570B54AD8
:103870001278D2B2B2498A700295AA1C9046032AE5
:1038800015DD0322AD498946AD4F0321C91A002336
:103890009A46631CDBB24846005DC0B2B854641857
:1038A000E2B2101D54463C541C004245F1DBFCF7CB
:1038B0004DFDA54B18701B78002B19D00023A34891
:1038C000802212049146A249002290469E4A9446C4
:1038D00082694F463A42FBD1CA5CD2B2026042468C
:1038E000CA540133DBB262461278D2B29342EFD3AC
:1038F0000022954B1A700132964B1A60029F0137D5
:10390000BE4225DD00221A608F490A7001321A601A
:1039100023009CE78A4BFE221A70F93A5A70002263
:103920009A708D480278D2B2511CC9B20170DA7017
:1039300086221A71843A5A71804AD278D2B29A7128
:10394000FCF704FD804B1870FCF79CFCFDF7FAFABD
:10395000824B1B78002B34D00022814B1A80814A85
:1039600001211D00804B9946A020C00580246400E1
:10397000592693681942FCD093680B4393602B88B7
:1039800001339BB22B802B889BB24B45F1D9162378
:103990009C46882706516346035107510359002B63
:1039A000F8D0724B98461B689C46032367463B43FE
:1039B00047463B606E4F6F4B1F6083680B438360CD
:1039C000D7E7684B9B68DB0700D44DE2654A9168F6
:1039D00001230B439360684B1B78002B04D0674A8C
:1039E00013780133DBB213705D4A138801339BB245
:1039F0001380634A13780133DBB21370614B1B7879
:103A0000002B6AD1604B1B78002B66D15F4B1A6884
:103A100001321A601A68FA235B009A4253D15C4B58
:103A200000221A700421597001399970DA7001323C
:103A30001A7108325A71574A80231B04916919423E
:103A4000FCD10020FCF74CFC524BD96810220A43F1
:103A5000DA60D96820220A43DA60D96808220A436A
:103A6000DA604B4B5B78012601244A4F80231B040C
:103A70009946474D00239846BB694A461342FBD1FD
:103A8000AB5DDBB23B60A85D019B5840C0B2FCF768
:103A90009FFB01904346AB550134E4B226006B789E
:103AA00001339C42E8DD3B4A80231B0491691942A3
:103AB000FCD1384B019A1A60012335490022CA54BF
:103AC00001333C2BFBD1314B1A68334B9A4204D95A
:103AD00001232C4A1370314A13702B4B1B78002B97
:103AE00000D096E1244B1B78002B00D0F9E02C4944
:103AF0000B78DBB25A1CD2B20A70032B00D8F0E06C
:103B000000230B701D4A1370264A13780133DBB271
:103B100013701378DBB2202B00D9C7E01378DBB227
:103B20001F2B00D9DDE013785A00D3189B001E4AE2
:103B3000D3189B7ADB0744D41A49ADE01401002066
:103B4000BC010020FD010020B10100200000054063
:103B50008C00002094420050BB0100207E00002019
:103B60003C030020200001401027000000C000504E
:103B70000400FA050CED00E0980100202906002061
:103B8000BC08002048030020F80200209401002017
:103B9000FC020020000015403075000042030020A8
:103BA00074060020A7040020A8040020BF4B1B7847
:103BB0005A00D3189B00BE4A944663449B7ADB07A5
:103BC0006AD5BA480378DBB2B9495C00E2189200C2
:103BD0008A1813890133138103785A00D3189B0084
:103BE000CB181A89C3235B009A4231D103785A005B
:103BF000D3189B00CB189A7A0124A2439A720378B7
:103C00005A00D3189B00CB1800221A81A94B1A70B6
:103C1000A94B1B68002B0BD0A84B1B78002B07D09F
:103C20000078C0B2FDF720F90022A54B1A7058E0C9
:103C30009E4B1A789E4851008A18920082180021E3
:103C400091721B785A00D3189B00C318596048E042
:103C5000964C23780133DBB29A4A13701078C0B2C5
:103C6000FCF73EFB23785A00D3189B00904AD318E8
:103C70009B7A5B0735D5904B1B68002B31D08F4B5F
:103C80001B78002B2DD0894B1878C0B2FDF7ECF8CB
:103C900000228B4B1A7024E00B780133DBB20B70DF
:103CA0000B78DBB21F2B00D880E71AE0814B1B7822
:103CB000002B0ED1844A80231B0491691942FCD148
:103CC0007E20FCF70DFB814A11684B424B4113608B
:103CD00004E00123794A13707D4A1370FF22734B6D
:103CE0001A707C4B1B78002B0AD07B4B1B88DB04A3
:103CF00003D50122794B1A6002E00022774B1A604B
:103D0000774A13780133DBB213701378002B37D165
:103D1000744B1B68002B05D1734A13780133DBB257
:103D2000137002E00022704B1A706F4B1B78022B4D
:103D300026D1684B1B78002B03D00022654B1A70EC
:103D400002E00122634B1A70684AFE231370FA3BAB
:103D500053700023937066480378DBB2591CC9B2D4
:103D60000170D370872313715A4B1B78591E8B41F6
:103D7000DBB25371FCF7EAFA5E4B1870FCF782FA7B
:103D80005D4A13780133DBB213705C4B1B68002B68
:103D900007D15B4B1B68002B03D15A4B1B68002BD0
:103DA00037D059490B889BB25A1C92B20A80574AA5
:103DB00093422ED90122564B1A70564A137801337A
:103DC000DBB213700021504B19801378DBB2092B42
:103DD0001FD90022494B1A60494B1A60494B1A609F
:103DE0004C4B1A70414BFE311970FA3959709A7068
:103DF0003F480278D2B2511CC9B20170DA708622F3
:103E00001A71563A5A71FCF7A1FA3A4B1870FCF73E
:103E100039FA414B1B68002B26D03F4B1A68013AF8
:103E20001A601B68002B1FD13C4B1B78002B1BD04A
:103E300000233B4A904600213A4A94463A4F3B4E73
:103E40003B4D3C4C354A91465A0040461152604623
:103E50001152D1539153515311530133DBB24A469E
:103E60001278D2B29A42EFD8334B1B78002B00D194
:103E700012E1324B1B78002B00D107E1304B1B784D
:103E8000DBB2532B60D002D84D2B05D0FBE06D2B5D
:103E900002D0732B58D0F6E001222A4B1A706C32F4
:103EA000124B1A70FCF7EAFAEDE0C046A7040020B6
:103EB000A8040020B2010020C00800204803002010
:103EC000FE010020FD010020000015406C42005062
:103ED000420300204B0300203C030020944200508A
:103EE00041030020904200502F060020BC0100201A
:103EF000BB010020B1010020BC080020040200200A
:103F0000880000209C01002000020020B80B000067
:103F10003006002077060020800000209901002054
:103F2000540100207C06002064030020D000002003
:103F30003406002008020020F80200207D00002046
:103F4000480200203F030020AA4B1B78002B57D0CB
:103F5000A9494B78303B1B01DBB2A84A13708B7820
:103F60001178303BCB18DBB213701378DBB2202B07
:103F700002D92022A14B1A709F49CB78303B1B01FC
:103F8000DBB29E4A53700B795178303BCB18DBB2D1
:103F900053705378DBB2202B02D92022974B5A70F2
:103FA00095494B79303B1B01DBB2944A93708B7976
:103FB0009178303BCB18DBB293709378DBB2202B37
:103FC00002D920228D4B9A708C490A784B788978D7
:103FD0009B18CB18DBB28A4D2B708A4C732323704D
:103FE00028780009FCF7EAF860702878C0B2FCF77E
:103FF000E5F8A0700D23E3700422834B1A7035E0BE
:104000007D4A5178C9B27D4B19709178C9B2597007
:10401000D278D2B29A701B78DBB2202B02D9202240
:10402000764B1A70754B5B78DBB2202B02D92022BD
:10403000724B5A70714B9B78DBB2202B02D9202235
:104040006E4B9A706D490A784B7889789B18CB181B
:10405000DBB26B4A13706B4B732119701278D2B2BA
:104060005A700D229A700A3A674B1A70FCF7D4F80E
:104070000122664B1A706832624B1A70FCF7FEF927
:1040800000225D4B1A700022614B1A705E4B1B7848
:10409000002B01D0FCF7C0F85E4B1B78DBB20A2B7B
:1040A00000D984E29B005C4AD3589F46544B1B784E
:1040B000002B02D10122594B1A700022584B1A7062
:1040C000564B1B78002B62D1564A916822330B4322
:1040D00093600122544B1A600022544B1A70544BC7
:1040E0001B78002B05D0464B1A780023002A05D1F7
:1040F00046E0504B1B78002BF5D141E04E4A9146EB
:104100004E484F4A92464F4F4F4E504D1A005C005A
:104110004946615A8846215A8C4641466C4621815F
:104120002489644505D04A49097801240C4348494B
:104130000C7054005146615A8846E15B8C464146FA
:104140006C4621812489644505D0414909780224BF
:104150000C433F490C705200945B525B9446A2B2F0
:10416000624506D03A4C22789446042261460A43BE
:1041700022700133DBB2224A1278D2B29A42C5D8F9
:10418000244A13780133DBB21370FEF7E4FF0622F2
:10419000204B1A70FEF7DFFF244B1B78002B01D158
:1041A000FEF7D9FF1F4A916844230B439360012215
:1041B000284B1A60264B1B78002B03D1264B1B780B
:1041C000002B0DD01B4B1B78002B02D069220D4B0E
:1041D0001A70FCF753F900231F4A13701C4A13701E
:1041E0000022124B1A700B4A13780133DBB21370A2
:1041F000FEF7B1FFCD00002048020020B8010020EA
:1042000099010020BC010020B10100203F030020E3
:104210007D00002049030020344E0000B30100203F
:10422000C50800208040005084420050BC08002097
:10423000A5040020F80200207C0600205401002084
:10424000D000002064030020080200203406002073
:10425000B40100208842005030060020E24B1B7859
:10426000DBB2032B01D8FEF776FFE04A93684421C6
:104270008B4393600023DE4A1360DB4A1370DD4BEF
:104280001B78002B2BD00022DB4DDC4B9846DC4CFE
:10429000DC4B9C46DC48DD4B9A46002153005E5BBC
:1042A0006F463E813E89B14646464F469F531E5B50
:1042B0006F463E813E89B14666464F469F531E5A21
:1042C0006F463E813E895746DE5359531953195262
:1042D0000132D2B2C74B1B78DBB29342DED8CC4B53
:1042E0001B68002B08D0CB4B1B78C3495B00585A86
:1042F0008022120202435A52C74B1B68002B08D07F
:10430000C44B1B78BE495B00585A802212020243FC
:104310005A52C24B1B68002B08D0BE4B1B78BA49BF
:104320005B00585A8022120202435A52BC4A137848
:104330000133DBB21370FEF70EFFAB4B1B78002B83
:1043400001D1FEF708FFA94A916811230B4393603E
:104350000122B44B1A600022A34B1A70B04A1378A2
:104360000133DBB21370FEF7F6FE9F4B1B78002B78
:1043700001D1FEF7F0FE9D4A936811218B439360B3
:104380000023A84A1360984A1370A54A1378013392
:10439000DBB21370FEF7DFFE934B1B78002B01D1CD
:1043A000FEF7D9FE914A936822218B439360002344
:1043B0009D4A13608C4A13700822994B1A70FEF7BD
:1043C000CAFE894B1B78002B01D1FEF7C4FE874A39
:1043D000916844230B4393600122854B1A600022AD
:1043E000814B1A708E4A13780133DBB21370FEF7DB
:1043F000B2FE7D4B1B78DBB2012B01D8FEF7ABFE82
:104400007A4A936844218B4393600020784B18606C
:10441000804A1378784C5B00195B4908195313786C
:10442000774C5B00195B49081953137876495B0098
:104430005A5A52085A526C4B1870754B1B68002B15
:1044400008D0744B1B786C495B00585A80221202CA
:1044500002435A52704B1B68002B08D06D4B1B78DF
:1044600067495B00585A8022120202435A526B4B32
:104470001B68002B08D0674B1B7863495B00585AB8
:104480008022120202435A52654A13780133DBB28A
:104490001370FEF760FE544B1B78002B01D1FEF722
:1044A0005AFE524A916844230B4393600122504BB9
:1044B0001A6000224C4B1A70594A13780133DBB250
:1044C0001370FEF748FE484B1B78DBB2012B01D876
:1044D000FEF741FE454A936844218B4393600020D8
:1044E000434B18604B4A1378434C5B00195B4908F7
:1044F00019531378424C5B00195B49081953137820
:1045000041495B005A5A52085A52374B1870404B77
:104510001B68002B08D03F4B1B7837495B00585A6B
:104520008022120202435A523B4B1B68002B08D0D8
:10453000384B1B7832495B00585A802212020243E2
:104540005A52364B1B68002B08D0324B1B782E4931
:104550005B00585A8022120202435A5233490B78A8
:10456000DBB25A1CD2B20A700D2B04D808222C4B95
:104570001A70FEF7F0FD2A4A13780133DBB213708C
:10458000FEF7E9FD184B1B78002B01D1FEF7E3FD88
:104590000022154B1A701F4A13780133DBB21370D7
:1045A0001F4A13780133DBB21370FEF7D4FD0E4BB4
:1045B0001B78002B01D1FEF7CEFD164B1B780D4A60
:1045C0001278DBB2934202D30022124B1A700022FF
:1045D000134B1A70FEF7BFFDFCF7B4FCFFF7B8F9F8
:1045E000FCF7B0FCFFF7B4F9BC0800208040005095
:1045F0008842005099010020540100207C060020D0
:1046000064030020D00000203406002008020020AF
:104610004C420050B30100205C4200508C420050DC
:10462000490300208042005084420050C508002009
:10463000304A13780133DBB213702F4B1B79DBB296
:10464000F02B01D0FFF7FAF84AE000222B4B9C46F2
:1046500050008118890061448C7A04231C43012393
:1046600023438B720023984600230B81224B5F79F2
:10467000FFB28418A400654667559E79F6B24E7065
:10468000DD79ECB200948C701C7A0C715C7A4C7100
:104690009C7A8C71DC7AE3B29A46CB71184B444613
:1046A0001C700C245C700B249C704446DC701C71E4
:1046B00070245C71541C6D462C722C7A9C71DF71D5
:1046C0001E72009C5C720D799D724979D9728118B5
:1046D000890061448979197351465973FEF797FF30
:1046E000054B9B780020002B01D0FFF7A5F8FEF7C3
:1046F0001BFFC046C608002014010020A8040020AB
:10470000FC02002010B53A4B1B68DBB2394A127824
:10471000D2B21F2A13D8374A1278002A0AD0354A53
:104720001278013A51008A18920033498A18002100
:10473000118104E00020BE2252002F4988522F4AE6
:104740001278002A23D1012B51D901212B4A117053
:104750002B490A789BB202329A18FF20024029485E
:1047600002800A78D2B2501CC0B2087026485200AB
:104770008024640014520A78D2B2541CE4B20C7043
:10478000520013520B785B0000221A522FE01C4A91
:1047900012781C490988914219D10024174A1470D3
:1047A00017490A78D2B2501CC0B208709BB21648A2
:1047B000520013520B78DBB25A1CD2B20A705B0063
:1047C000802292001A520B785B001C520FE00C49B9
:1047D0000A78D2B2501CC0B208709BB20A4852008C
:1047E00013520B785B0000221A52084B1A7010BD4E
:1047F00000001540FD010020A804002098010020C1
:10480000C408002074000020BC06002029060020F7
:10481000F0B583B0664B1B68DBB26A46D371654B5B
:104820001B78002B00D1AAE0634B9B78002B17D09C
:10483000012B00D0B9E0604BD9784A1CDA706B4686
:10484000DA1DDB79DBB25D48435413780D2B00D0C1
:10485000ABE00022584B9A700132594B1A70A4E019
:104860006B4607331B784D3BDAB2292A00D99CE00E
:104870009300544AD3589F46534A544B1A6001221E
:104880004D4BDA706B4607331B78DBB24B490B702C
:104890004B4B1A7089E04C4A4C4B1A6001234C4A2E
:1048A00013704549CB706A4607321278D2B243483A
:1048B00002708B7079E0474A137859424B41DBB262
:1048C00013707421444B197013785A1E934130337E
:1048D000414A53700D2393700322404B1A7064E0D9
:1048E0003D4B56221A706521597072209870283AF3
:1048F000DA7031241C715A7130259D71DC71023CD3
:104900001C7213345C7239359D724426DE721D733D
:104910005C73153C9C730A35DD730C3E1E745E742B
:104920009C741C34DC7425341C7506345C759975D4
:10493000D8750C38187629365E7603389876D9768D
:10494000453919774C3C5C7798773A38D8775427B3
:104950005F54333FDE554C373F3E9F5501369D55E2
:104960004F3D5955213505315D54273501315D5491
:1049700001315A54213A1A55184B187015E0184B4A
:104980001A78D2B2511CC9B2197069460731097838
:10499000C9B2144881541A78D2B2002181541B78CC
:1049A000002B02D10122104B1A7003B0F0BDC0469B
:1049B00000000540F802002074000020480200209A
:1049C0007D000020704E0000A086010080000020C5
:1049D00076060020CD000020BC010020B10100209F
:1049E00085000020A40300208400002010B582B0C0
:1049F0000422204901A800F023F91F4B1B6A002064
:104A0000A022D202134216D11A0301D41B4800E09F
:104A10001B489A030FD4DA05D20D023280085043A6
:104A20001A04920F01A9895C9B04DB0E02335943DF
:104A300000F07AF88000134B18600F4B1B690722B7
:104A40001340022B03D09B000A4AD31858680A4B24
:104A50009B690F211940013100F066F8094C606034
:104A6000094B9C466044094900F05EF8A06002B022
:104A700010BDC046184F000000020050001BB700D8
:104A8000008051010000002020A1070040420F00DB
:104A900030B500221E4B1A601E4B1B6907321340B3
:104AA0000DD11D4A1B4B1A621C4B1A48042102E00F
:104AB000013B002B23D0C2681142F9D01FE0072B25
:104AC00025D1174A134B1A62164B1248042102E0F3
:104AD000013B002B13D0C2681142F9D00FE0D55032
:104AE000D450D050D1580029F9D00222094B1A6174
:104AF000002180235B00A022D205D15007E0A02234
:104B0000D20580235B00592516248820E7E730BDB5
:104B1000000000200002005017420000E12E0000BB
:104B20003956080067560000002243088B4274D3B0
:104B300003098B425FD3030A8B4244D3030B8B429E
:104B400028D3030C8B420DD3FF22090212BA030CA7
:104B50008B4202D31212090265D0030B8B4219D388
:104B600000E0090AC30B8B4201D3CB03C01A5241A8
:104B7000830B8B4201D38B03C01A5241430B8B42F0
:104B800001D34B03C01A5241030B8B4201D30B03D9
:104B9000C01A5241C30A8B4201D3CB02C01A524100
:104BA000830A8B4201D38B02C01A5241430A8B42C3
:104BB00001D34B02C01A5241030A8B4201D30B02AC
:104BC000C01A5241CDD2C3098B4201D3CB01C01AC6
:104BD000524183098B4201D38B01C01A52414309D0
:104BE0008B4201D34B01C01A524103098B4201D3BE
:104BF0000B01C01A5241C3088B4201D3CB00C01A2B
:104C0000524183088B4201D38B00C01A52414308A2
:104C10008B4201D34B00C01A5241411A00D20146C7
:104C2000524110467047FFE701B5002000F006F83A
:104C300002BDC0460029F7D076E770477047C046EE
:104C400070B50F2A32D90C0004430B00A40731D1F0
:104C500015000400103D2D0901352D0149191E686C
:104C600026605E6866609E68A660DE681033E66057
:104C700010349942F3D10F2345191340032B1BD94C
:104C80001C1F0023A4080134A400CE58EE500433A6
:104C90009C42FAD103232D1909191A4005D000238B
:104CA000CC5CEC5401339A42FAD170BD0500002A65
:104CB000F5D1FAE70500F2E71A00F8E7061D000053
:104CC000FA120000DC150000B4160000A81600005F
:104CD00006160000521600007E160000DE170000C7
:104CE0004E1C00002618000038130000D8130000E6
:104CF0002A130000201C0000061D0000C81600003A
:104D000012170000F4160000061D00009E1A000095
:104D1000741A00004C1800007C190000921C00005E
:104D20006E1B0000E8120000061D0000061D0000BA
:104D3000061D0000061D0000061D0000061D0000E7
:104D4000061D0000061D0000061D0000061D0000D7
:104D5000061D0000061D0000061D0000061D0000C7
:104D6000061D0000061D0000061D0000061D0000B7
:104D7000061D0000061D0000061D00008A1C000024
:104D80008A1C0000842A0000BE1D0000F41D0000E3
:104D90002E1E0000241E0000381E0000921E00007F
:104DA000241F0000541F0000842A0000A21F0000DE
:104DB000842A0000842A0000842A0000842A00003B
:104DC000842A0000B62400008E250000F024000094
:104DD000A4270000842A0000842A0000842A0000FE
:104DE000842A0000842A00002C230000CE1F00002B
:104DF000842A0000842A0000842A0000842A0000FB
:104E0000842A0000B6280000282A0000282A000072
:104E1000282A0000842A0000FA2900001C2600002D
:104E20005226000090260000C6260000042700003D
:104E30003A270000AC400000984100005C420000AE
:104E40003A4300006A43000098430000C243000058
:104E5000F243000096440000C64400008445000070
:104E6000001BB7000000000000000000008051019E
:104E700078480000AA490000AA490000AA49000099
:104E8000AA490000AA49000096480000B648000060
:104E9000AA490000E0480000AA490000AA49000011
:104EA000AA490000AA490000AA490000AA49000036
:104EB000AA490000AA490000AA490000AA49000026
:104EC000AA490000AA490000AA490000AA49000016
:104ED000AA490000AA490000AA490000AA49000006
:104EE000AA490000AA490000AA490000AA490000F6
:104EF00078480000AA490000AA490000AA49000019
:104F0000AA490000AA49000096480000B6480000DF
:104F1000AA490000E048000001020204001BB7009B
:104F20000000000080F0FA021027000000000000DE
:0C4F3000000000000000000000805101A3
:0C4F3C0080F0FA0280F0FA02320000005F
:00000001FF
